:1000000090F8037492F075F8FF75E8FF7590FF9013
:10001000F8007400F0A3F0A3F0780079007A007B78
:100020000020B30302800012008930B203120046A0
:1000300012003580ECC3C2D2C2B4C2B5E89AFCE962
:100040009BFD12005722C3C2D2C2B4C2B5E82AFC3B
:10005000EB39FD120057228C90ED90F802F092B42B
:1000600030D21BD2B520E70B7408120098742B1203
:100070000098227408120098742D120098227408B7
:1000800012009874201200982290F800E0F9A890CD
:1000900090F801E0FBAAE822F599C2993099FD2277
:00000001FF
